:0300000002001EDD
:03000B000201F3FC
:10001B000201B875812078087400F608E8B420F85E
:10002B00750D01758921D2B9758B1A758D1AD28E02
:10003B00D2ABD2AF900244120050C2B77514FAE59E
:10004B001470FC80EFC0028583108582117A0085C5
:10005B001083851182EA93F8EA0493F58288837002
:10006B0003E860071200790A0A80E4D00222C0027A
:10007B00E493A3700302012FFA54F0B4E008EA549E
:10008B000FF50802012CB4002EC083C082EA540F76
:10009B00B40105900234800AB4020590023C800240
:1000AB00800D78157908E493F608A3D9F9800280BE
:1000BB0006D082D083806AB4F007EA540FF5128021
:1000CB0060B4D00FEA3132E5874401F587E50D6066
:1000DB00F6804EEA3132EAC39410C4540FF8E508A7
:1000EB0075F00CA428C083C082C333F8900170C292
:1000FB008CD29493F58CF509E80493F58AF50AC232
:10010B008D751403E51470FCD2A9D28CD082D083E8
:10011B00E5874401F587E50D60F6C2A9D29480010D
:10012B00EA02007BD00222540FC333F8C083C08293
:10013B0090015293C2ABF50BE80493F50CD2AB755F
:10014B000D00D082D083220180012000C0009000DE
:10015B006000400030002000180012000C00090065
:10016B000600050003FDFFFE1CFE37FE52FE6AFE75
:10017B0082FE98FEADFEC0FED3FEE4FEF5FF04FF4B
:10018B0013FF21FF2EFF3AFF45FF51FF5BFF65FF7A
:10019B006EFF77FF7FFF87FF8EFF95FF9CFFA2FF10
:1001AB00A8FFADFFB3FFB7FFBCFFC0FFC5C0D0C0FA
:1001BB00E0E50E6005150E0201EE750E04E5146008
:1001CB00021514E50F6004150F801885120FE50C4E
:1001DB006004150C800DE50B7005750D0180041581
:1001EB000B150CD0E0D0D032C0D085098C850A8A93
:1001FB00C28DD28CC0E0C000051EE51E30E002B2FD
:10020B00947815E513C31392D528F8E6A2D54001CF
:10021B00C4540FF8E59054F048F590E51304540FCF
:10022B00F513D000D0E0D0D0327CFC720279A975E6
:10023B0045789ABCDEF01234560250025302530238
:10024B006E029C000001F500E2452816E1B696B659
:10025B00E216E196B8E21828E1B8E215E1B8E196AA
:10026B00869400E1B5E21826E1B6E2152846E1B620
:10027B00E2182846688896866644452816E1B696A5
:10028B00B6E216E196E268686868452816E1B6940E
:03029B0000D2008E
:00000001FF
